:1000000062C07DC57BC07AC079C078C077C076C039
:1000100075C074C073C072C071C070C06FC06EC054
:100020006DC06CC06BC005010904A1010901A100EC
:1000300085010930093115002502750895028102F4
:10004000150025019506750105091901290681028A
:10005000950275018101C0C0040309041A037700E9
:10006000770077002E0061007200740065006D005B
:100070002E00720075001C03550053004200200042
:10008000440041004E004300450020005000410064
:1000900044001201100100000008424232E1040055
:1000A0000102000109022200010100801909040077
:1000B00000010300000009210101000122320007B4
:1000C00005810308000F11241FBECFE5D4E0DEBF79
:1000D000CDBF10E0A0E6B0E0E4E9FDE002C005908D
:1000E0000D92AA3BB107D9F710E0AAEBB0E001C02E
:1000F0001D92AC3FB107E1F73ED04AC681CF9C01CB
:10010000E199FECF3FBB2EBB6DBB0FB6F894E29AD0
:10011000E19A0FBE0895FC0180818076803249F516
:100120008181813031F58281882321F48091BA0068
:1001300083708F5F8093BA008091BA00E3E08E9F56
:10014000F0011124E354FF4F8093BB00DF018D9138
:100150008093BC0081818093BD0011968C91809327
:10016000BE008BEB90E09093E1008093E00084E090
:10017000089580E008952F923F924F925F926F9280
:100180007F928F929F92AF92BF92CF92DF92EF9227
:10019000FF920F931F93DF93CF93CDB7DEB7C9576D
:1001A000D0400FB6F894DEBF0FBECDBFDE0157962C
:1001B000E0EBF0E088E001900D928150E1F7DE0184
:1001C0005F96E8EAF0E088E001900D928150E1F757
:1001D00080E2898380E18A8388E08B8384E08C835A
:1001E000DE01D396ECE9F0E08CE001900D928150B5
:1001F000E1F7DE01DF96E0E9F0E08CE001900D929E
:100200008150E1F7DE011B96EAE8F0E086E001901C
:100210000D928150E1F7DE01A55BBF4FEEE7F0E004
:100220008CE001900D928150E1F7DE01A95ABF4F99
:10023000E2E7F0E08CE001900D928150E1F7DE0101
:10024000AD59BF4FE6E6F0E08CE001900D92815091
:10025000E1F7DE015196E0E6F0E086E001900D92D4
:100260008150E1F7E199FECF80E390E09FBB8EBB28
:10027000E09A2DB3E1962FAFE1972F3F19F4E19665
:100280001FAEE19740E050E020E030E0A3E38A2E8B
:10029000912C8C0E9D1EFBE0AF2EB12CAC0EBD1E22
:1002A000EFE3CE2ED12CCC0EDD1E7BE4E72EF12C1D
:1002B000EC0EFD1E8E010F5E1F4FBE01695A7F4F6F
:1002C000F401E20FF31F0190F081E02D9081D50140
:1002D000A40FB51F8C91892B8083F601E20FF31FC9
:1002E0000190F081E02D90818C918095892380830D
:1002F000F701E20FF31F0190F081E02D9081D8010A
:10030000A40FB51F8C91809589238083FB01E20F98
:10031000F31F0190F081E02D90818C9180958923CD
:1003200080834F5F5F4F2E5F3F4F4630510541F650
:10033000BE01695E7F4FAE01415E5F4F20E030E05D
:100340008E010F5F1F4FDB01ED91FD91BD0190818B
:10035000D801A20FB31F8C91892B8083FA01E19001
:10036000F190AF01F70190818C9180958923808372
:100370002F5F3F4F2430310531F7FE01359686E07F
:10038000DF011D928A95E9F79E01295D3F4FE896AE
:100390003FAF2EAFE8978CE0D9011D928A95E9F71F
:1003A000A598AD9A12BE83B7856083BF2F8D38A103
:1003B000E6963FAF2EAFE6978BA19CA1E4969FAF48
:1003C0008EAFE49729A03AA04DA05EA0E2961FAEA2
:1003D000E29766247724DE011B96EA96BFAFAEAFA4
:1003E000EA975E010894A11CB11CFE013596DE015E
:1003F000979611921D921D92EA962EAD3FADEA9707
:10040000E217F307B1F781E08093C0008093C10049
:100410008091C200807C8093C20020D28B989398F8
:1004200088E893E1E0E9F1E03197F1F70197D1F73E
:100430008B9A939A78948824992410E0DD24CC2414
:10044000E0961FAEE09761E0E62EF12C14D2809189
:10045000D10084FF5CC0E114F104E1F549853A85DF
:100460002D815F819E816885E1968FADE19788231C
:1004700099F041708091C2008C7F3170330F842BD2
:10048000832B8093C2002F5F251B2093C0009F5FAA
:10049000961B9093C1001EC021708091C2008C7F7A
:1004A0009170990F822B892B5170550F550F837FB7
:1004B0006170660F660F660F852B862B4170429523
:1004C000407F8F7C31703295330F307E842B832BAD
:1004D0008093C2008091BA0083708F5F8093BA00CE
:1004E00093E0899FF0011124E354FF4F8093BB00F8
:1004F000DF018D918093BC0081818093BD001196B6
:100500008C918093BE0064E08BEB90E0BDD2E096CE
:10051000AFADE097A13041F0A13018F0A23089F5DD
:1005200010C09D9B28C02DC00894611C711CB9EEA1
:100530006B16B3E07B0628F1E2E0E096EFAFE097C0
:1005400020C09D9B1EC081E0E196FFADE197F8279A
:10055000E196FFAFE197E199FECF80E390E09FBB8A
:100560008EBBE1962FADE1972DBB0FB6F894E29AC2
:10057000E19A0FBE3ACF31E0E0963FAFE0976624B4
:100580007724123091F1133034F4112359F01130E3
:1005900009F05AC10FC0133009F442C0143009F0F9
:1005A00053C154C012BE8824992411E0E2961FAEB4
:1005B000E2974AC1AE01415C5F4F20E030E0FA01B2
:1005C000A191B191AF019C91EBE0F0E0EC0FFD1F28
:1005D000E20FF31F8081809589238C932F5F3F4F1B
:1005E0002630310561F712E02FC1AD2DB0E0FD01DD
:1005F000EE0FFF1F23E630E02C0F3D1FE20FF31F2D
:100600000190F081E02D8081E1E1F0E0EC0FFD1F31
:10061000AE0FBF1F9C91892309F016C113E014C1CE
:10062000AD2DB0E0FD01EE0FFF1FEA0DFB1D06AC86
:10063000F7ADE02D80812BE030E02C0F3D1FA20FA5
:10064000B31F9C91892B808314E0FEC0AD2DB0E0D8
:10065000AD01440F551FE3E6F0E0EC0FFD1FE40F82
:10066000F51F0190F081E02D8081E1E1F0E0EC0FD9
:10067000FD1FEA0FFB1F9081892309F4E5C082B7B3
:10068000E2963FADE2973F5FE2963FAFE2973134AB
:1006900014F411E0D9C0382D2227280F311DE114A0
:1006A000F10409F497C00894E11CF11C89E5E816EF
:1006B00082E0F80608F44AC0F501E40FF51F86A1B0
:1006C00097A18217930710F437A326A3C70169E106
:1006D00070E04AD3892BD1F5E1969FADE19799233C
:1006E00001F1CC2079F0E696AEADBFADE6978C91E6
:1006F000998189278C93E496EEADFFADE4978081D4
:100700009B8108C0D1018C919A8189278C93F20139
:1007100080819C8189278083C394F1E0FC15A8F037
:1007200015C0AC2DB0E0FD01EE0FFF1FEA0DFB1D63
:10073000068CF78DE02D8081AA0DBB1D9C91892729
:100740008083C39423E02C1508F4CC2439EBE31602
:100750003BE0F30608F470C087E2E82EF12CEC0EC3
:10076000FD1E00E010E0D7012D913C91C90165E02C
:1007700070E0FAD2620F731FF701619371937F01EA
:100780004FE750E0C801DBD20E5F1F4F0C30110560
:1007900051F7E696AEADBFADE6979C918981809505
:1007A00089238C93F10190818A81809589238083AC
:1007B000E496AEADBFADE4979C918B818095982374
:1007C0009C93F20190818C81809589238083EE2413
:1007D000FF2432C04A0D5B1DFA0186A197A1821742
:1007E0009307A8F4E5E0F0E0EC0FFD1FEA0FFB1F14
:1007F00021E0208333E03D15F8F0FA01268D378D96
:10080000F9018081AA0DBB1D9C91892B14C0E5E0E4
:10081000F0E0EC0FFD1FEA0FFB1F1082F3E0FD1567
:1008200058F0FA01268D378DF9019081AA0DBB1D74
:100830008C91809589238083D394F5E0FD1518F47D
:1008400010E0DD2401C010E008B600FEFFCD88B73F
:10085000816088BF0894811C911CF8CD85B78360A6
:1008600085BF8BB780648BBF8BE48093D2008AE511
:100870008093D10008951F93CF93DF939091E2006E
:10088000935097FDA6C02091DF008091DE008D324D
:1008900009F09DC0983009F09AC0CCE0D0E0C21BAE
:1008A000D109CA51DF4F83EC8093C6008AE580935B
:1008B000B8001092BF008881807621F0CE012BDC39
:1008C000282F7CC09A811092CF008981882321F43F
:1008D0001092D00022E06CC0853019F49093E300B0
:1008E00066C0863009F04FC08B81813041F482E9C7
:1008F00090E09093E1008093E00022E140C08230DC
:1009000041F484EA90E09093E1008093E00022E2D9
:1009100036C08330F9F48A81882341F488E590E079
:100920009093E1008093E00024E029C0813041F4FD
:100930008CE590E09093E1008093E0002AE11FC0F5
:100940008230E1F486E790E09093E1008093E0004C
:100950002CE115C0813241F486EB90E09093E100E8
:100960008093E00029E00BC0823241F486E290E0FF
:100970009093E1008093E00022E301C020E080E456
:100980008093BF001BC0883021F421E085EE90E009
:1009900011C0893019F49093E50009C08A3011F430
:1009A00021E006C08B3019F48BE48093D20020E064
:1009B0008FEC90E09093E1008093E0008F8188239A
:1009C00021F48E81821708F4282F2093B900109209
:1009D000E2008091B80084FF49C08091B9008F3F48
:1009E00009F444C0182F893008F018E0811B809367
:1009F000B9008091C60098E889278093C60011232A
:100A000041F12091E0003091E1008091BF0086FF2C
:100A10000DC0A7ECB0E080E090E0F901E80FF91F0D
:100A2000E491ED9301961817C1F708C0912FD901F1
:100A3000E7ECF0E08D9181939150E1F71150812F17
:100A400090E01F5F0196820F931F9093E1008093C7
:100A5000E000612F87EC90E04ED0612F6C5F6C302E
:100A600019F08FEF8093B9006093B8009AE080B3DB
:100A7000847131F49150D9F71092E3001092DD00A7
:100A8000DF91CF911F9108951F93DC01162F809164
:100A9000D10084FF07C08091D20098E88927809315
:100AA000D20003C08AE58093D100912FE3EDF0E0FE
:100AB0008D91819391501916DCF3612F83ED90E0B5
:100AC0001AD01C5F1093D1001F910895A82FB92F41
:100AD00080E090E041E050EA60956F5F58F42D911E
:100AE00038EF82279795879510F0842795273F5FE9
:100AF000C8F3F3CF0895EADF8D939D930895CF93C4
:100B0000CFB7CF93DF93849BFECF849B0BC0849B96
:100B100009C0849B07C0849B05C0849B03C0849B41
:100B200001C08BC06F93C091DF00DD27CA51DF4F3A
:100B30002F9365E5849B03C02F916F91E6CF0F93B0
:100B40001F934F9320E040E15F9300B3047104FBD7
:100B500027F93F9350E03BE039C0147140642F7790
:100B6000012F53501EC0406810B314712F7753509B
:100B70001FC0406400B32F770471D1F153500000BF
:100B800023C0406210B32F77147191F153500000CD
:100B900025C004711027515012F45D5F0000115000
:100BA00027952C3F10B3C8F61471012701502795E3
:100BB0002C3FC8F64227499300B3047110274F73A6
:100BC000115027952C3FA8F64695469510B3147101
:100BD00079F00127015027952C3F98F66B5A60F366
:100BE000315000B3B0F600C010E41ABF002719C09E
:100BF0003B503195C31BD04010E41ABF0881033C21
:100C000009F10B34F9F02091DD001981110F121355
:100C1000EDCF4A81441F093651F10D3211F0013EEA
:100C200029F70093E4003F915F914F911F910F913D
:100C30002F916F91CAB7C6FD66CFDF91CF91CFBF1D
:100C4000CF9118950091E400002369F31091E20020
:100C5000112391F5343092F13093E2000093DE00DD
:100C60001091DF003BE0311B3093DF0027C0009183
:100C7000E20001300CF50AE54F7049F43091B800FC
:100C800034FD1DC00093B800C6ECD0E01CC030910C
:100C9000D10034FD14C00093D100C2EDD0E013C0E8
:100CA000052710E000C0000002BB1AC0052710E0B5
:100CB000221F1DC010E021C04AE502C032ED432FC3
:100CC000C4E1D0E032E011B31461949A02B311BBD5
:100CD00054E120E865E320FF052702BB279517951F
:100CE0001C3FF0F66695B8F7B1F720FF052702BB69
:100CF000279517951C3FD0F62795179517FF0527C1
:100D000000001C3F02BBB0F629913A9519F70B7E03
:100D10001091E300110FC651D04002BB11F01093A7
:100D2000DD0010E41ABF006111B31B7E402F4B7E23
:100D300054E05A95F1F702BB11BB42BB74CFDF926E
:100D4000EF92FF920F931F93D72E7A018C01FA0135
:100D500009956D2DC8010196F70109951F910F9115
:100D6000FF90EF90DF900895AA1BBB1B51E107C0D5
:100D7000AA1FBB1FA617B70710F0A61BB70B881F2B
:100D8000991F5A95A9F780959095BC01CD010895BA
:040D9000F894FFCF05
:100D9400011004028020300033003300360030009C
:100DA40030003200350035003800320032003100A6
:100DB40034003400370031003100020802010140E0
:100DC400320035003500350038003200310034007F
:100DD400340034003700310038003800380038005F
:0A0DE40037003700370037005AFFD0
:00000001FF
